:10000000830100308A00C328FF0003088301D70062
:100010000408D8000A08D9008A015008E0005108F5
:10002000DE005208E1005308DF005408E4005508E0
:10003000E2005608E3005C08DA005D08DB0083019B
:100040008C1D672883168C1D672883128C118316DC
:10005000941A2C288312A2018316141D3B288312A4
:100060002108483E8400831300089300A10A07304A
:10007000A1051416632883121308BD00A20A2208E2
:10008000023A031D47283D080739A10063280330C1
:100090002202031C6328210B4E28A0152108023AD6
:1000A000031920162108063A031D5828A801A80A9A
:1000B00007302102031862282108483E8400831378
:1000C0003D088000A10A8A1552248A1114138B1945
:1000D0000B1CA52883120608BF000B102306BE00C8
:1000E000C0390319A3283E1B3F1B832810100F089B
:1000F000C1000E08C00020100C189228A016C400E1
:100100004108C5009228BE1BBF1B922810100F0883
:10011000C3000E08C20020100C1892282017C60039
:100120004308C7003F1B3E1F9728201C9C28BF1B6D
:10013000BE1FA3282018A32804308E008F010C10A6
:100140003130900020143F08A30083120C182010B7
:100150006008D0005E08D1006108D2005F08D300BB
:100160006408D4006208D5006308D6005A08DC0091
:100170005B08DD005808840059088A00570883008E
:10018000FF0E7F0E0900213084004430DA20203039
:1001900084002130DA2083010730DD00F430DC00F8
:1001A000443084005030DE2083018A111E2F040663
:1001B0008001840A0406031DD7280034D0008A1168
:1001C000EB208A118000840A0408500603190034C9
:1001D000DF288312DC00DD1BF6285D1BFE285D088E
:1001E0008A005C08DC0A0319DD0A820083135D18AB
:0C01F00083175C08DC0A8400000808008B
:100DBC0083013C08D1003B08D000BC1F0800D009BF
:100DCC00D109D00A0319D10A080083120313D401E4
:100DDC00D5010310D30CD20C031CFB2E5008D407E6
:100DEC0051080318510AD5070310D00DD10D520824
:100DFC00530403190034EF2E613083019F000C3033
:100E0C0097009D008030831692007C3083129200F4
:100E1C00183083168700FC308600FF3085009F0158
:100E2C00433081000B178B17831295019B0108002F
:100E3C000227672FB030831693008A155F24B230D7
:100E4C00831693008A155F24B430831693008A1599
:100E5C005F24B630831693008A155F24B83083164E
:100E6C0093008A155F24BA30831693008A155F2489
:100E7C00BC30831693008A155F24BE308316930012
:100E8C008A155F248A159725AA01AA0A8A1537267E
:100E9C008A15C226AA01AA0A8A150623A0178A1542
:100EAC00C226AA01AA0AA0178A1506230230AA0094
:100EBC008A1537260230AA00A0178A1506238A1134
:100ECC00662F06083C39D200D3019D2F5208031916
:100EDC00202F043A0319252F0C3A03192A2F043A10
:100EEC0003192F2F1C3A0319342F043A0319392FE5
:100EFC000C3A03193E2F043A0319432F3C3A0319B9
:100F0C00482F043A03194A2F0C3A03194E2F043A6E
:100F1C000319502F1C3A0319542F043A0319572F55
:100F2C000C3A03195C2F043A0319602F662F5308EF
:100F3C0003196C2F662F83120313D601D11FAD2F0B
:100F4C00D009D00A0319D103D1095617D617530863
:100F5C008039D606D31FBB2FD209D20A0319D3036B
:100F6C00D309BB2F83120313D601D401D501520828
:100F7C005304031DC42FD001D10100341F30D604FB
:100F8C000310D60AD20DD30D031CC72FD30CD20CD1
:100F9C0053085102031DD42F52085002031CDC2F9E
:100FAC005208D0025308031C530AD102D40DD50D9C
:100FBC00D60BD61ACC2FD61FE82FD409D40A031976
:100FCC00D503D5095408D2005508D300561F003458
:100FDC00D009D00A0319D103D10900347734013474
:100FEC0077340134003400340034003400340034DD
:040FFC000034003489
:1011DA000B1D50290B1152243408803AD0002E08D6
:1011EA00803A5002031DFB282D0833028312031391
:1011FA0003180329B30A0319B40A15292E08803AD9
:10120A00D0003408803A5002031D0D2933082D02FC
:10121A0003181629FF3083120313B307031CB40300
:10122A00A01652243608803AD0003008803A50027C
:10123A00031D21292F0835028312031303182929B4
:10124A00B50A0319B60A3B293008803AD000360895
:10125A00803A5002031D332935082F0203183C290E
:10126A00FF3083120313B507031CB6032017522459
:10127A004B08FF3C810034082E06031D462933081B
:10128A002D06031D502936083006031D4E29350840
:10129A002F060319A0108301080052243308BB004B
:1012AA003408BC008A11DE263608D3003508D2007D
:1012BA008A11EB265408D0005508D1007D30D2009F
:1012CA000030D3018A11A1278A155408B90055089C
:1012DA00BA003908B41F80293302B1003A08031C46
:1012EA003A0A3402B20039083307AB003A08031845
:1012FA003A0A34078E293307B1003A0803183A0A22
:10130A003407B20039083302AB003A08031C3A0A20
:10131A003402AC003208803AD000803050027C306F
:10132A0003193102031CAC292C08D1002B08D00068
:10133A003108D002031CD1033208D1027B30500796
:10134A00AB000030031801305107AC00C62932083F
:10135A00803AD0007F3050028530031931020318D9
:10136A00C6298530D000FF30D1003108D002031CD5
:10137A00D1033208D1025008AB070318AC0A51084E
:10138A00AC072C08803AD000803050027C30031918
:10139A002B02031CE3293208D1003108D0002B08A4
:1013AA00D002031CD1032C08D1027B305007B100B4
:1013BA000030031801305107B200FD292C08803A89
:1013CA00D0007F305002853003192B020318FD2903
:1013DA008530D000FF30D1002B08D002031CD10386
:1013EA002C08D1025008B1070318B20A5108B207F3
:0613FA003208803AD00029
:10140000803050027C3003193102031C0B2A7B30E0
:10141000B100B201192A3208803AD0007F30500260
:101420008530031931020318192A8530B100FF30C5
:10143000B2002C08803AD000803050027C30031972
:101440002B02031C272A7B30AB00AC01352A2C0869
:10145000803AD0007F305002853003192B020318E8
:10146000352A8530AB00FF30AC00522C52243508B1
:101470003307B10036080318360A3407B2003508BE
:101480003302AB003608031C360A3402AC003208C3
:10149000803AD000803050027C3003193102031CA6
:1014A000642A2C08D1002B08D0003108D002031C7C
:1014B000D1033208D1027B305007AB000030031853
:1014C00001305107AC007E2A3208803AD0007F30CC
:1014D000500285300319310203187E2A8530D0006E
:1014E000FF30D1003108D002031CD1033208D102F1
:1014F0005008AB070318AC0A5108AC072C08803A17
:10150000D000803050027C3003192B02031C9B2A30
:101510003208D1003108D0002B08D002031CD103BF
:101520002C08D1027B305007B10000300318013085
:101530005107B200B52A2C08803AD0007F30500203
:10154000853003192B020318B52A8530D000FF30EF
:10155000D1002B08D002031CD1032C08D102500863
:10156000B1070318B20A5108B2073208803AD00016
:10157000803050027C3003193102031CC32A7B30B7
:10158000B100B201D12A3208803AD0007F30500237
:101590008530031931020318D12A8530B100FF309C
:1015A000B2002C08803AD000803050027C30031901
:1015B0002B02031CDF2A7B30AB00AC01ED2A2C0888
:1015C000803AD0007F305002853003192B02031877
:1015D000ED2A8530AB00FF30AC00522C83018C101B
:1015E0002508C83A031D042BA6080319FC2AA708DE
:1015F0000319FC2AA901002BA901A90A2017A0168A
:10160000A701A601A5010800A50A08000B108B156B
:1016100052248C18A01F0D2BEE22A01A112B201F74
:10162000082BA01A182B202B4408B3004508B4003F
:1016300045083406031D1E2B44083306031D142BD6
:10164000201B272B2F2B4608B5004708B60047085C
:101650003606031D2D2B46083506031D232BC60118
:10166000C7014608C4004708C500201344182017C6
:1016700083120313A012201BA0163408803AD00056
:10168000823050022630031933020318A02B34088D
:10169000803AD00080305002C93003193302031C55
:1016A000A02BA601A60A8930B3070318B40AFE309E
:1016B000B407B41F752BD001D10133085002B70015
:1016C0003408031C340A5102B800380DB80CB70CAA
:1016D000380DB80CB70CD001D10137085002B70053
:1016E0003808031C380A5102822B3408D100330811
:1016F000D000510DD10CD00C510DD10CD00C500894
:10170000B7005108B8003708B3070318B40A3808FF
:10171000B4073408803AD0007F305002FF300319FC
:101720003302031C9F2B3408803AD00080305002D3
:1017300002300319330203189F2BB301B401522462
:101740003608803AD0008230500226300319350224
:101750000318032C3608803AD00080305002C9307C
:1017600003193502031C032CA701A70A8930B5070A
:101770000318B60AFE30B607B61FD82BD001D10128
:1017800035085002B7003608031C360A5102B8006B
:10179000380DB80CB70C380DB80CB70CD001D1010E
:1017A00037085002B7003808031C380A5102E52BED
:1017B0003608D1003508D000510DD10CD00C510D98
:1017C000D10CD00C5008B7005108B8003708B50745
:1017D0000318B60A3808B6073608803AD0007F30BA
:1017E0005002FF3003193502031C022C3608803AE0
:1017F000D000803050020230031935020318022C49
:10180000B501B6015224A60803193E2CA7080319F6
:101810003E2C2A08023A031D102C36228A15122C5F
:1018200052218A1552243208803AD000803050026A
:101830000130031931023108031C232CB900013097
:1018400048248610282C003CB90001304824861416
:1018500052242C08803AD000803050020130031905
:101860002B022B08031C392CB90002304824061027
:101870003E2C003CB900023048240614A908031984
:10188000082BB90101304824B90102304824082B43
:101890008301BA003A0B4F2C39089500080039082B
:1018A0009B0008008301A40803195A2CC03087004C
:1018B000A401080021308700A401A40A08004630D2
:1018C0008316031381008030940036308312940015
:1018D0008316910183128C1183168C150A308312A2
:1018E000CF005224A019762C201EBE2CA01D792CCE
:1018F000A016201E7C2C2017A01120125224C808EC
:1019000003198A2C4808023A03198A2C4808043A19
:10191000031DA12C8030D000FF30D10049085007B2
:10192000AD0051080318510AAE008030D000FF30DE
:10193000D1004A085007AF0051080318510AB000FF
:10194000AB2C4908AD00AE01AD1BAE034A08AF0099
:10195000B001AF1BB0035224C8080319B12C480BC7
:10196000B62C4B08FF3C8100A014BE2C2D08B30000
:101970002E08B4002F08B5003008B600C8080319B7
:10198000C62C480B422DA808031D422DA01CC92CB3
:10199000ED205224A01E052D3408803AD00080305E
:1019A0005002013003193302031CE62C5224861026
:1019B0003408803AD000803050027C300319330262
:1019C0000318F22C3308AB003408FF2C5224861481
:1019D0003408803AD0007F3050028530031933023A
:1019E0000318F62C7B30AB00AC01002DD001D101E7
:1019F00033085002AB003408031C340A5102AC0017
:101A00002B08B90001304824A0125224201F892D30
:101A10003608803AD0008030500201300319350278
:101A2000031C222D522406103608803AD000803044
:101A300050027C300319350203182E2D3508B100F1
:101A400036083B2D522406143608803AD0007F30E9
:101A500050028530031935020318322D7B30B10056
:101A6000B2013C2DD001D10135085002B100360839
:101A7000031C360A5102B2003108B9000230482472
:101A80002013892D06304802A80803188A2D031D4B
:101A9000892DA01A4D2D201F892D52244808043A63
:101AA0000319562D4808053A031D592D36228A156B
:101AB0005B2D52218A1552243208803AD0008030A2
:101AC00050020130031931023108031C6C2DB9009A
:101AD000013048248610712D003CB90001304824A3
:101AE000861452242C08803AD000803050020130F5
:101AF00003192B022B08031C822DB9000230482445
:101B00000610872D003CB90002304824061420132B
:101B1000A012A8080319712CA801B90101304824AA
:101B2000B90102304824A0112012A010712CC3303A
:101B300083160313810052241F199B2D201DEA2DAB
:101B40008130D000FF30D1001E085007B30051088B
:101B50000318510AB40061309F0020115224340848
:101B6000803AD0008030500202300319330234082A
:101B7000031CCB2D803AD000803050027C300319FA
:101B80003302031CC52D7B30C62D3308B90001304C
:101B900048248610342E803AD0007F305002FF3027
:101BA000031933020318E72D3408803AD0007F3040
:101BB00050028530031933020318E02D7B30E22DEB
:101BC0003308003CB900013048248614342EB90192
:101BD0000130332E8130D000FF30D1001E08500775
:101BE000B50051080318510AB60059309F0020155E
:101BF00052243608803AD000803050020230031957
:101C000035023608031C152E803AD0008030500271
:101C10007C3003193502031C0F2E7B30102E350843
:101C2000B900023048240610342E803AD0007F30AC
:101C30005002FF30031935020318312E3608803A5E
:101C4000D0007F30500285300319350203182A2E48
:101C50007B302C2E3508003CB90002304824061495
:101C6000342EB9010230482452241F159B2DC33055
:101C700083160313810052241F193B2E201D662E4C
:101C80008130D000FF30D1001E085007B30051084A
:101C90000318510AB400A1309F0052243408803A3E
:101CA000D0007F305002FF3003193302031C642E32
:101CB0003408803AD00080305002023003193302D9
:101CC0000318642EB301B40120118B2E8130D00093
:101CD000FF30D1001E085007B50051080318510A03
:101CE000B60099309F0052243608803AD0007F30E9
:101CF0005002FF3003193502031C8A2E3608803A41
:101D0000D0008030500202300319350203188A2EA9
:101D1000B501B60120152A08023A031D922E36227B
:101D20008A15942E52218A1552243208803AD00006
:101D3000803050020130031931023108031CA52EF6
:101D4000B900013048248610AA2E003CB9000130A9
:101D50004824861452242C08803AD0008030500247
:101D6000013003192B022B08031CBB2EB9000230D3
:101D700048240610C02E003CB90002304824061446
:101D80001F153B2E0B108B1552248C18A01FC92E2B
:101D9000EE22A01AD02E642F4408B3004508B400E8
:101DA00045083406031DD62E44083306031DCC2EE9
:101DB000C401C5013408803AD00082305002263078
:101DC0000319330203185D2F3408803AD0008030A5
:101DD0005002C93003193302031C5D2FA601A60A65
:101DE0008930B3070318B40AFE30B4075224B41F75
:101DF000132FD001D10133085002B7003408031C5F
:101E0000340A5102B800380DB80CB70C380DB80CB4
:101E1000B70CD001D10137085002B7003808031CB5
:101E2000380A5102202F3408D1003308D000510D58
:101E3000D10CD00C510DD10CD00C5008B70051086A
:101E4000B8003708B3070318B40A3808B407A9085C
:101E500003192C2FB301B4013408803AD00080302C
:101E600050020130031933023408031C492F803A11
:101E7000D000803050027C3003193302031C432F02
:101E80007B30B300B4013308B90001304824861018
:101E90005C2F803AD0007F30500285300319330226
:101EA0000318562F8530B300FF30B4003308003CD0
:101EB000B9000130482486145224A9080319632F5D
:101EC000B90101304824A012201B6B2FC42E4608F4
:101ED000B5004708B60047083606031D712F4608AF
:101EE0003506031D672FC601C7013608803AD000AA
:101EF000823050022630031935020318F82F3608B5
:101F0000803AD00080305002C93003193502031CDA
:101F1000F82FA701A70A8930B5070318B60AFE30C3
:101F2000B6075224B61FAE2FD001D101350850029A
:101F3000B7003608031C360A5102B800380DB80C39
:101F4000B70C380DB80CB70CD001D10137085002CE
:101F5000B7003808031C380A5102BB2F3608D100DD
:101F60003508D000510DD10CD00C510DD10CD00C36
:101F70005008B7005108B8003708B5070318B60A6B
:101F80003808B607A9080319C72FB501B6013608E6
:101F9000803AD000803050020130031935023608F3
:101FA000031CE42F803AD000803050027C300319AB
:101FB0003502031CDE2F7B30B500B6013508B900B1
:101FC000023048240610F72F803AD0007F305002AC
:101FD0008530031935020318F12F8530B500FF3025
:101FE000B6003508003CB9000230482406145224DB
:101FF000A9080319FE2FB901023048242013C42E6A
:02400E00723FFF
:00000001FF
